:0C0000000EC0FECFFDCF44C0FBCFFACFF6
:10000C00F9CFF8CFF7CFF6CF0000020004001400B0
:10001C000000F894EE27ECBBE5BFF8E1A4B7A77F8E
:10002C00A4BFF1BDE1BD8DE0A2E0ED938A95E9F7A7
:10003C0080E4A0E6ED938A95E9F7E6E1F0E0C89557
:10004C003196802DC8953196902D0097B9F0C895B2
:10005C003196A02DC8953196B02DC8953196102C9F
:10006C00C89531966E2F7F2FF02DE12DC8953196C6
:10007C000D920197D9F7E62FF72FE1CFEFE9EDBFFE
:10008C00C0E730C06A937A93AA93EA93FA93EFB7D6
:10009C00EA93E0E0E2BFA0E7C3D0EF5FFF4F6F4F02
:1000AC007F4FC3D0E991EFBFF991E991A991799173
:1000BC0069911895BFD000E00E3140F47AD01E2F14
:1000CC0078D0E11709F000E00F5FF6CFE12FB5D043
:1000DC000895BB9AC398E8EEF3E0FA93EA9394D0B0
:1000EC00BB980895E0E8E6BDE0E0E6BDE8BBE0E1E2
:1000FC00E7BBE0E0EFBDE5E0E3BFE0E0E2BFE6BF79
:10010C00E9BDEBBFE5BFE2E0E9BFE0E8E8B9E0E05C
:10011C00E3B9E4BBE6B9E9E3E1BDE9E2E1BD78941A
:10012C002197E0E0E883A895C5DFE883E42DF52D61
:10013C00309739F4E881E170E13011F4C49A40D081
:10014C0035C0E130A0E0FA0789F4E881E17069F488
:10015C0045D0AA3AE0E0BE07E0E08E07E0E09E075B
:10016C0010F445D002C0B5DF2BD020C0E230A0E0A7
:10017C00FA07E1F433D0A938E7E7BE07E0E08E07D1
:10018C00E0E09E0708F033D0E881E170E13071F4D3
:10019C00A0DFE1E0F0E04E2E5F2EE0E0E093700097
:1001AC00E0937100E0937200E09373002196B8CF56
:1001BC00FFCF8AEC98E00197F1F7E6B3E170089570
:1001CC00E1E0F0E04E0E5F1EE0E0E0937000E093A3
:1001DC007100E0937200E09373000895A091700099
:1001EC00B091710080917200909173000895442435
:1001FC005524E0E0E0937000E0937100E09372000E
:10020C00E0937300C4980895E991F991309639F010
:10021C008AEC98E00197F1F7A8953197C9F7089502
:10022C00ED91FD916D917D9108957E936E93FE936A
:10023C00EE9308951A930A930895099119910895CC
:00000001FF
